:020000040000FA
:080000000002040000000000F2
:020000040000FA
:040008009A04000056
:020000040000FA
:04000C009A04000052
:020000040000FA
:040010009A0400004E
:020000040000FA
:040014009A0400004A
:020000040000FA
:040018009A04000046
:020000040000FA
:04001C009A04000042
:020000040000FA
:040020009A0400003E
:020000040000FA
:040024009A0400003A
:020000040000FA
:040028009A04000036
:020000040000FA
:04002C009A04000032
:020000040000FA
:040030009A0400002E
:020000040000FA
:040034009A0400002A
:020000040000FA
:040038009A04000026
:020000040000FA
:04003C009A04000022
:020000040000FA
:040040009A0400001E
:020000040000FA
:040044009A0400001A
:020000040000FA
:040048009A04000016
:020000040000FA
:04004C009A04000012
:020000040000FA
:040050009A0400000E
:020000040000FA
:040054006004000044
:020000040000FA
:040058007E04000022
:020000040000FA
:04005C009A04000002
:020000040000FA
:040060009A040000FE
:020000040000FA
:040064009A040000FA
:020000040000FA
:040068009A040000F6
:020000040000FA
:04006C009A040000F2
:020000040000FA
:040070009A040000EE
:020000040000FA
:040074009A040000EA
:020000040000FA
:040078009A040000E6
:020000040000FA
:04007C009A040000E2
:020000040000FA
:040080009A040000DE
:020000040000FA
:040084009A040000DA
:020000040000FA
:040088009A040000D6
:020000040000FA
:04008C009A040000D2
:020000040000FA
:040090009A040000CE
:020000040000FA
:040094009A040000CA
:020000040000FA
:040098009A040000C6
:020000040000FA
:04009C009A040000C2
:020000040000FA
:0400A0009A040000BE
:020000040000FA
:0400A4009A040000BA
:020000040000FA
:0400A8009A040000B6
:020000040000FA
:0400AC009A040000B2
:020000040000FA
:0400B0009A040000AE
:020000040000FA
:0400B4009A040000AA
:020000040000FA
:0400B8009A040000A6
:020000040000FA
:0400BC009A040000A2
:020000040000FA
:0400C0009A0400009E
:020000040000FA
:0400C4009A0400009A
:020000040000FA
:0400C8009A04000096
:020000040000FA
:0400CC009A04000092
:020000040000FA
:0400D0009A0400008E
:020000040000FA
:0400D4009A0400008A
:020000040000FA
:0400D8009A04000086
:020000040000FA
:0400DC009A04000082
:020000040000FA
:0400E0009A0400007E
:020000040000FA
:0400E4009A0400007A
:020000040000FA
:0400E8009A04000076
:020000040000FA
:0400EC009A04000072
:020000040000FA
:0400F0009A0400006E
:020000040000FA
:0400F4009A0400006A
:020000040000FA
:0400F8009A04000066
:020000040000FA
:0400FC009A04000062
:020000040000FA
:040100009A0400005D
:020000040000FA
:040104009A04000059
:020000040000FA
:040108009A04000055
:020000040000FA
:04010C009A04000051
:020000040000FA
:040110009A0400004D
:020000040000FA
:040114009A04000049
:020000040000FA
:040118009A04000045
:020000040000FA
:04011C009A04000041
:020000040000FA
:040120009A0400003D
:020000040000FA
:040124009A04000039
:020000040000FA
:040128009A04000035
:020000040000FA
:04012C009A04000031
:020000040000FA
:040130009A0400002D
:020000040000FA
:040134009A04000029
:020000040000FA
:040138009A04000025
:020000040000FA
:04013C009A04000021
:020000040000FA
:040140009A0400001D
:020000040000FA
:040144009A04000019
:020000040000FA
:040148009A04000015
:020000040000FA
:040208009A04000054
:020000040000FA
:04020C009A04000050
:020000040000FA
:040210009A0400004C
:020000040000FA
:040214009A04000048
:020000040000FA
:040218009A04000044
:020000040000FA
:04021C009A04000040
:020000040000FA
:040220009A0400003C
:020000040000FA
:040224009A04000038
:020000040000FA
:040228009A04000034
:020000040000FA
:04022C009A04000030
:020000040000FA
:040230009A0400002C
:020000040000FA
:040234009A04000028
:020000040000FA
:040238009A04000024
:020000040000FA
:04023C009A04000020
:020000040000FA
:040240009A0400001C
:020000040000FA
:040244009A04000018
:020000040000FA
:040248009A04000014
:020000040000FA
:04024C009A04000010
:020000040000FA
:040250009A0400000C
:020000040000FA
:040254009A04000008
:020000040000FA
:040258009A04000004
:020000040000FA
:04025C009A04000000
:020000040000FA
:040260009A040000FC
:020000040000FA
:040264009A040000F8
:020000040000FA
:040268009A040000F4
:020000040000FA
:04026C009A040000F0
:020000040000FA
:040270009A040000EC
:020000040000FA
:040274009A040000E8
:020000040000FA
:040278009A040000E4
:020000040000FA
:04027C009A040000E0
:020000040000FA
:040280009A040000DC
:020000040000FA
:040284009A040000D8
:020000040000FA
:040288009A040000D4
:020000040000FA
:04028C009A040000D0
:020000040000FA
:040290009A040000CC
:020000040000FA
:040294009A040000C8
:020000040000FA
:040298009A040000C4
:020000040000FA
:04029C009A040000C0
:020000040000FA
:0402A0009A040000BC
:020000040000FA
:0402A4009A040000B8
:020000040000FA
:0402A8009A040000B4
:020000040000FA
:0402AC009A040000B0
:020000040000FA
:0402B0009A040000AC
:020000040000FA
:0402B4009A040000A8
:020000040000FA
:0402B8009A040000A4
:020000040000FA
:0402BC009A040000A0
:020000040000FA
:0402C0009A0400009C
:020000040000FA
:0402C4009A04000098
:020000040000FA
:0402C8009A04000094
:020000040000FA
:0402CC009A04000090
:020000040000FA
:0402D0009A0400008C
:020000040000FA
:0402D4009A04000088
:020000040000FA
:0402D8009A04000084
:020000040000FA
:0402DC009A04000080
:020000040000FA
:0402E0009A0400007C
:020000040000FA
:0402E4009A04000078
:020000040000FA
:0402E8009A04000074
:020000040000FA
:0402EC009A04000070
:020000040000FA
:0402F0009A0400006C
:020000040000FA
:0402F4009A04000068
:020000040000FA
:0402F8009A04000064
:020000040000FA
:0402FC009A04000060
:020000040000FA
:040300009A0400005B
:020000040000FA
:040304009A04000057
:020000040000FA
:040308009A04000053
:020000040000FA
:04030C009A0400004F
:020000040000FA
:040310009A0400004B
:020000040000FA
:040314009A04000047
:020000040000FA
:040318009A04000043
:020000040000FA
:04031C009A0400003F
:020000040000FA
:040320009A0400003B
:020000040000FA
:040324009A04000037
:020000040000FA
:040328009A04000033
:020000040000FA
:04032C009A0400002F
:020000040000FA
:040330009A0400002B
:020000040000FA
:040334009A04000027
:020000040000FA
:040338009A04000023
:020000040000FA
:04033C009A0400001F
:020000040000FA
:040340009A0400001B
:020000040000FA
:040344009A04000017
:020000040000FA
:040348009A04000013
:020000040000FA
:100400006FE72100AE7E22000E0188000000000090
:10041000000020000000E000020032000001200087
:100420002002880014000700440107000000E000DB
:1004300003003A00A07A26000100200002003700E5
:100440000000200001002000810F70000100320038
:1004500014000700000020000000E000020032004D
:10046000000002000000000008760200000000000A
:100470000040DA000000FE004440A900C03920001E
:100480000000E0000300320000002000A00188000E
:100490004440A800000006008A1F78008B1F7800E7
:1004A0000000060091018800800478000000EB0045
:1004B0001A003700E284440032A0B4009905BA0063
:1004C000E284440032A0B4009906BA00E2844400F9
:1004D00032A0B4000006EB00476FDE00FD07B2005B
:1004E000636CE10003003A00EBFF07000000EB0043
:1004F0000A003700606CE10004003A00005DEB0088
:100500008B05E900FDFF3E00040037006168E10053
:10051000010032000086EB000B00070019C7BA008B
:100520001905BA000E04E00003003A000A00E000DA
:10053000E0FF3A0000000600FE07B2009E018800BE
:100540008A047800F5FF3700395DBA008B05E900B1
:100550000C003200295DBA008B05E900080032006A
:100560000C00E00003003A00E284440032A0B40032
:10057000F5FF370019DDBA008B05E900FAFF3A00F4
:100580008904E800E184440032A0B40000000600C1
:10059000000000000000000000000000000000005B
:1005A000000000000000000000000000000000004B
:1005B000000000000000000000000000000000003B
:1005C000000000000000000000000000000000002B
:1008C000809FBE00821F780032118000204080008F
:1008D00001408000827078000408EC00204088000D
:1008E0000208E30001003A009560A9008560A900B4
:1008F0004F0178004F00BE0000400600809FBE0000
:100900000808EC00404088000A08E30002003A00B2
:100910009580A900040037003140800061407800D4
:100920000080FB00201188008580A9004F00BE00D8
:10093000004006000040DA000000FE000000050054
:1009400003F0A200889FBE008A9FBE008C1F780023
:100950004A010700510133006450E1004F003200AA
:100960006420E1005200320003826C0007003B006B
:100970000905D0000306D000820F54000C065D006C
:100980000200390002003200890178000306780075
:100990008582550004003D000003FD008103FD0039
:1009A0008502EA008B854200840F720002003B0042
:1009B00060001000E08018006011B8000005EB0036
:1009C0007A28E1000A00390006007800C75DDD00E2
:1009D000F707B200878075002D0037008281710013
:1009E0000A017800610560008180D1000080D30099
:1009F0008502E900F9FF3B000604400087844800B7
:100A000002003B0060041400E0841C000988A3007D
:100A1000070032008A8171008281710061016400E7
:100A20008904D1000884D3008B05E8001700370043
:100A30000978A30013003A000B00E0001300340013
:100A40008B05E9000804440089844C000A447400C2
:100A50000978A3000D003A000B00E0000700340005
:100A60008B05E9000804440089844C0001003A0029
:100A70000B0020000978A300F7FF32000001EB0013
:100A800002003700828171000A017800C00007006F
:100A90000CF0A70001F0A000090137006420E1007C
:100AA00002003A00838F6C00090133000801BE0088
:100AB0000200BE0002013700889FBE008A9FBE0070
:100AC0008C1F7800ED000700F400330003866C00F3
:100AD0006450E1002E0032006420E1003300320057
:100AE0006150E1002F0032006120E100310032004E
:100AF00085855500EB07B0000900200008042000A0
:100B0000050037000804440089844C000A003100C5
:100B10000603430087834B000001530081815B0083
:100B2000F8FF33000203BE000800A00008044400E0
:100B300089844C00F6FF3900C639DD00830173005B
:100B400001003200130020008904D1000884D30082
:100B50000998A300050032000800A7000300A000C8
:100B60008904D1000884D3008B05E8008904D100F2
:100B70000884D3000001EB000281D200840007004A
:100B800001F0A1000CF0A70001F0A000CC0037009C
:100B90006420E100CE0032000801BE000200BE0069
:100BA000F7FF37006120E100C90032006000B800A3
:100BB000F3FF37000000200001F82700F0FF3700A6
:100BC00014002000B0013700F4FF2F00AE01370001
:100BD0000003BE00940007006011B8000470A70075
:100BE00007F0A10007F8A30017003A006509B1005B
:100BF0000D0032000D003500860220000628E100BD
:100C000003003500030028006000B8000200050062
:100C100000004000818048000201490083814900B2
:100C20008502E900FAFF3A0000000600F88F420052
:100C3000050034008100D1000080D3008502E80067
:100C4000FCFF3A00000006006011B8008000EB00D5
:100C5000000005000001BE00730007000470A7003B
:100C600003F0A10003F8A30013003A006509B100E6
:100C700010003200090035006928E100020035004B
:100C800001002800000005000000400081804800AD
:100C90008502E900FCFF3A0000000600F88F4200E0
:100CA000050035008100D1000080D3008502E800F6
:100CB000FCFF3A00000006008000EB000000050089
:100CC0004F89DE00820178008A013700889FBE00CC
:100CD0008A9FBE00008270000402710004827100CD
:100CE000260032000004BE000200BE006011B80001
:100CF0006B092000950220000182CF000A00390014
:100D00000541B1000082CF00070039000541B10064
:100D10000982CF00040039000541B1000882CF00EC
:100D2000010039000541B1000542520012003200B5
:100D30000A003B0082817100610164008100D100E2
:100D40000080D3008984D3000884D3008B05E80099
:100D50000442E800F7FF3A000700370008044400A7
:100D600089844C0000004800818048008B05E90020
:100D70000442E900F9FF3A00050007004F05BE00F4
:100D80004F04BE00000006006011B800CFFF37001E
:100D900081002000618055000B003D000B00200009
:100DA00061FE2F000100E1001D003400828171000E
:100DB000610164008904D1000884D3000000E800C8
:100DC000FAFF3A0071002000610064000300700027
:100DD000020060000900320061044400E0844C001D
:100DE0000988A500050032008B05E8006808E100CD
:100DF00002003A008904D1000884D300F20F2000D9
:100E00000258E10005003D00C75DDD00F907B200B2
:100E10008980750008007800000006000BF82700A4
:100E20008B00780000000500C70ADE00F107B20061
:100E3000F50FB20008003200E1CF4200020032009C
:100E40000170A00024000500810F70000100320035
:100E50000408050044000500810F700002003A00FC
:100E6000140005008502E9000000400081C0480030
:100E7000FCFF3B000170A000240005000004BE0040
:100E8000E9FF07000003BE000405BE000200BE002B
:100E9000E5FF0700844F7500000006000200BE0059
:100EA0006450E100050036006420E10002003600D5
:100EB0000968A30001003A000800BE000160A0001C
:100EC0004F0678004F05BE004F04BE00000006002C
:100ED000F0FF2F00F1FF2700F9FF3700889FBE00C9
:100EE0008A9FBE008C1F7800E4FF0700EBFF3300F1
:100EF00003866C006450E100240032006420E100AD
:100F0000270032006150E100220032006120E10040
:100F1000210032008B854200EB07B1000134B8009C
:100F2000003AB8000804420089844A00013AB80037
:100F30000030B8008880400009014A0004003300F6
:100F40000000400081804800020149008B05E90053
:100F5000C909DD0083017000010032001300200088
:100F6000C814DE004814DD004709DE001200B2009C
:100F7000C808DE000884700085FF070001F0A100AA
:100F80000CF0A70001F0A000CDFF37006120E100C8
:100F9000CFFF32000801BE000200BE00F7FF37009D
:100FA0006150E100FCFF3A00C9FF37006022B80041
:100FB000060220000000D0008180D2000482D2000E
:100FC0008582D2000000A0000202520083825A00F3
:100FD000030031000202420083824A000000A100A7
:100FE0000603E900F3FF3A0000000600EFFF0700E8
:100FF0000400BE0000000600889FBE008A9FBE005D
:1010000030044200B0844A0030054B0090854B000C
:101010006000B1000898BE000A90BE000440E100E4
:1010200005C8E10006D0E10007D8E1000200310068
:10103000680040001008E8004F05BE004F04BE00E5
:1010400000000600889FBE008A9FBE003004BE00DC
:101050002005BE000418540005985C0006185D00C9
:1010600007985D00110020000440E10005C8E10080
:1010700006D0E10007D8E100010039008000EB0054
:10108000108810004F05BE004F04BE00000006008F
:101090001200FA00889FBE008A9FBE008C9FBE008F
:1010A000E0B79F00F1B79F0082BF9F0093BF9F00F2
:1010B0000605BE000404BE000000EB00D0B79F0090
:1010C000C0B79F00B0B79F00A0B79F0090B79F0028
:1010D0000006EB005FB19700CFB09700820141009E
:1010E0003FB097000200E00004003D003700070019
:1010F0007E805700C0FF0700030037003300070061
:101100007E805700CFFF0700DFB697000D00E0009C
:101110000C0035006FB29700FFB297000FBB97002D
:101120009FBB970010002000010020006011B80054
:1011300000027200818272000203730083837300D5
:101140001B0007000C06E80001042000810F560078
:10115000E0FF3A000D00E00004003D000802BE0080
:101160000A03BE007E805700A3FF07005FA8970018
:101170000000E00005003A001FB29700AFB29700F0
:101180003FB39700CFB39700090007006FB09700F7
:10119000FFB097000FB997009FB997004F06BE00A8
:1011A0004F05BE004F04BE000080FA00000006009C
:1011B0000100070000000600A4B79F00B5B79F001C
:1011C000C6B79F00D7B79F00000006004F09DE009A
:1011D00082817100B3B79F004F01DE008180400023
:1011E00082807000A1B79F008FB097004F09DE008A
:1011F000000040000200700090B79F007FA8970099
:101200004F01DE00818040008280700081B79F0026
:101210000D0007004F3ADE0000004000040070009F
:10122000F0AF9F00080007000402420085824A00D8
:1012300006034B0087834B00DFFF07000802BE0058
:101240000A03BE00000006002FB29700BFB297004D
:101250004FB39700DFB3970000000600881F7800A7
:1012600018002000881F780089FF07008F87E90099
:101270004F04780000000600801FEB0084FF070089
:101280008F87E90000000600889FBE008A9FBE008D
:10129000841F7800F9FE07004F007800110033002A
:1012A000F0FF2F00838F6C0006003B0004056500F3
:1012B0000A00A7000800370009F0A600100020006F
:1012C00008003700820F5400838F5C000300390050
:1012D0001000200001003E000000200009F0A700DF
:1012E0000000EA004F05BE004F04BE000000E00011
:1012F00000000600881F7800030478000300E00067
:1013000007003D0060001000E08018006001190037
:10131000E081190002003B0001F02D0003003700BE
:101320006AFE070008F0A70001F0A0004F04780053
:10133000000006008001780002003700B1597800F3
:101340000201E9000200E000FCFF3A000000060094
:101350008001780002003700815978000201E9001D
:0C1360000200E000FCFF3A000000060064
:020000040000FA
:10136C000052000045540000555200004E00000091
:10137C00525500004E0000004C4900005354000030
:10138C000045000058490000540000004E45000084
:10139C00570000004C450000540000004946000076
:1013AC0000540000484500004E000000454C000071
:1013BC0053450000004700004F5400004F00000050
:1013CC00474F0000535500004200000052450000FA
:1013DC004D00000050520000494E00005400000027
:1013EC00494E00005055000054000000464F0000CC
:1013FC0052000000544F0000004E00004558000001
:10140C00540000005245000041440000004400001C
:10141C0041540000410000005354000041520000B0
:10142C00545200000053000054410000525400007C
:10143C0000530000544F00005052000000530000B5
:10144C00544F000050000000534500004E44000073
:10145C00005200004543000045490000564500007D
:10146C00004300004C4B00000044000041540000BD
:10147C000042000049540000524500004144000065
:10148C00004100004443000000410000555800009A
:10149C00504900004E000000505300005500000061
:1014AC00505500004C4C000055500000004400000A
:1014BC00454C000041590000004100005558000007
:1014CC000046000052450000510000004455000049
:1014DC0054590000004D000041430000524F0000E1
:1014EC00004500004E44000000000000D0890000C0
:1014FC00D4890000D7890000DC890000E189000054
:10150C00E6890000B7890000EC890000F089000032
:10151C00F6890000FC890000008A0000038A0000A4
:10152C00088A00000D8A0000128A0000198A000047
:10153C001F8A0000258A00002A8A00002F8A0000DA
:10154C00378A00003B8A00003F8A0000478A00006F
:10155C004B8A0000528A0000568A00005D8A000007
:10156C00638A0000678A00006C8A0000718A0000A0
:10157C00778A000000000000002E0000003A0000F6
:10158C0020000000005E0000BCE20000613F000093
:10159C00DD830000C29C00007E200000A3FD000043
:1015AC001F4100009DC30000217F0000FCA2000031
:1015BC00401E00005F010000E3BD00003E60000023
:1015CC0082DC0000237D00009FC10000421C000053
:1015DC00FEA00000E1BF00005D03000080DE000003
:1015EC003C620000BEE00000025C0000DF810000F5
:1015FC00633D00007C220000C09E00001D430000E3
:10160C00A1FF000046180000FAA400002779000092
:10161C009BC5000084DA000038660000E5BB0000C2
:10162C0059070000DB85000067390000BAE40000B0
:10163C000658000019470000A5FB000078260000A2
:10164C00C49A0000653B0000D9870000045A0000D2
:10165C00B8E60000A7F900001B450000C698000082
:10166C007A240000F8A60000441A000099C7000074
:10167C00257B00003A64000086D800005B05000062
:10168C00E7B900008CD20000306E0000EDB3000012
:10169C00510F00004E100000F2AC00002F71000042
:1016AC0093CD0000114F0000ADF30000702E000030
:1016BC00CC920000D38D00006F310000B2EC000022
:1016CC000E500000AFF10000134D0000CE90000052
:1016DC00722C00006D330000D18F00000C52000002
:1016EC00B0EE0000326C00008ED00000530D0000F4
:1016FC00EFB10000F0AE00004C12000091CF0000E2
:10170C002D730000CA94000076280000ABF5000091
:10171C001749000008560000B4EA000069370000C1
:10172C00D58B000057090000EBB5000036680000AF
:10173C008AD4000095CB000029770000F4AA0000A1
:10174C0048160000E9B70000550B000088D60000D1
:10175C00346A00002B75000097C900004A14000081
:10176C00F6A80000742A0000C8960000154B000073
:10177C00A9F70000B6E800000A540000D789000061
:10178C006B35000049090000004F00000900000003
:10179C0048090000004C0000090000003E00000059
:1017AC00001B00005B000000440000004300000030
:1017BC000D0A00002800000078000000293E0000FF
:1017CC00002E000020000000427500007320000075
:1017DC005069000072610000746500002076000002
:1017EC0033000000436F00006D6D0000756E00004B
:1017FC00697400007920000046690000726D0000D9
:10180C00776100007265000020760000372E000022
:10181C00312000002D200000676F00006F2E0000AB
:10182C00676C00002F670000437A0000516E0000C7
:10183C005720000000290000002E0000203C000072
:10184C00000000000000000001000000000000008B
:10185C000200000000000000040000000000000076
:10186C000800000000000000100000000000000054
:10187C0020000000000000004000000000000000FC
:10188C00800000000000000080000000000000004C
:10189C000001000000000000000200000000000039
:1018AC000004000000000000000800000000000020
:1018BC0000100000000000000020000000000000EC
:1018CC00004000000000000000800000000000004C
:1018DC0000000000010000000000000002000000F9
:1018EC0000000000040000000000000008000000E0
:1018FC000000000010000000000000001434000084
:10190C00040D00008206000040030000A00100004E
:10191C00CF0000006700000044000000220000001F
:10192C007F00000000000000000000002C010000FF
:10193C00000000005802000000000000B00400008D
:10194C00000000006009000000000000C012000050
:10195C00000000008025000000000000403800005E
:10196C0000000000004B0000000000008070000030
:10197C00000000000096000000000000C0DA00002B
:10198C000000000000E100000000000000C20000A8
:10199C000100000000F400000100000000E800005D
:1019AC000300000030300000302C0000003000003C
:1019BC0030000000080800000808000008000000C3
:1019CC0000300000313200003334000035360000A6
:1019DC003738000039410000424300004445000004
:1019EC0046000000314100004C5300000142000051
:1019FC0050760000330000002100000000100000B1
:101A0C0000230000000F00004240000040050000D1
:101A1C00410200000000000000000000006900000E
:101A2C00D05D00006DDB00005D6B0000CB5D000045
:101A3C0069D000005D00000000000000181C0000D0
:101A4C001D0C0000161A00000B0F00001E170000E2
:101A5C001B000000145000000108000001030000EE
:101A6C000000000000200000290000009D2500005F
:101A7C000D000000003500003F6200006100000016
:101A8C002900000000000000000000000000000021
:081A9C00000000000000000042
:020000040000FA
:101AA4002208EC000080FB00E1CA2100E14078003C
:101AB4008100FB0080072000808F5000100032005E
:101AC40074005000808F5000090032000080E9004B
:101AD400808F5000080032000040EB0072072000A5
:101AE400828F500008003A003000200005003700C3
:101AF4001000200003003700200020000100370000
:101B04000000EB000040E8000000060042168000E0
:101B140080006100B0BC28000100320080BC2800B5
:101B24007027070000000600521680008000610044
:101B340010BD280001003200E0BC2800692707001E
:101B4400000006008000780000C3B3000100E0003C
:101B5400010032000040E800AE2607000000060045
:101B640070ED80002008E30003003A0070C0B30069
:101B7400A8260700070037000000E800F20F200045
:101B8400E1DA210082086000208E28000100200094
:101B94005833070000000600608D28000100200073
:101BA4005433070030E621001081FB0000032000BD
:101BB4000091B90061AC21000100410049270700F0
:101BC40040E6210010007800640060000300320049
:101BD400A07C2800010020004633070040BD2800F7
:101BE4004027070000000600889FBE008A9FBE00B1
:101BF400800578001141800000418000808F5000F2
:101C04000C003200E4CA21008041EB00F20F2000F6
:101C1400037278000000E90002006000808F500029
:101C2400FBFF3A00004188000041EB00E1CA2100BB
:101C3400827078000B00E9000080FB000241800004
:101C44000004EB00820F500012003200E1CA2100B0
:101C5400E14078000104E00007003A000300370087
:101C6400E44078000104E00005003A000000E800C8
:101C74000084FB0007003700F30F2000E4CA2100B2
:101C84000000E90003006000820F5000F4FF3A00F6
:101C94000004EB00C0FF07008B0F54000D0032005E
:101CA400E9CA2100FA0F200069407C005926070088
:101CB4000041800068F07C000000E8008A006000B9
:101CC400014188000804E8000A046400888F550074
:101CD400F5FF3A00004180000041EB00E1CA210019
:101CE4008270780070ED88004F05BE004F04BE007E
:101CF40000000600889FBE008A9FBE001841800035
:101D04000804E9000884FB0000418000880F5000AB
:101D1400170032000005EB00E9CA21000BDB2100AB
:101D240069407C000004E0000C003A000800E9006F
:101D34000080FB00694078000004E00007003200E6
:101D44000A05E8001B007800800F550003003600E8
:101D5400800DE80008007800A3FF07000804E900EC
:101D64000884FB0000418000880F5000ECFF3A001B
:101D740070C0B300272607004F05BE004F04BE0005
:101D840000000600889FBE008A9FBE0019418000A3
:101D94008904E9008984FB0000418000890F500018
:101DA400180032008000EB00EACA21000BDB21009E
:101DB4006AC07C000004E0000D003A000900E9005C
:101DC4000080FB006A4078000004E0000800320054
:101DD4008100E8001B04E900810F540004003A006C
:101DE400880D7800090078007FFF070088007800DC
:101DF4008904E9008984FB0000418000890F5000B8
:101E0400EBFF3A0080ED8000E10F50000300320048
:101E140070C0B300FF250700140037005EFF070001
:101E24000041800011418000810F50000900320000
:101E3400E4CA21008041EB00F20F20000372780015
:101E44000000E90002006000808F5000FBFF3A00B0
:101E5400004188000041EB00E1CA21008270780053
:101E640070ED880000DB21000008EB004F05BE0088
:101E74004F04BE000000060011C0B30030DB210097
:101E8400014878008000EB0081ED8800004180006B
:101E9400E2CA2100017178000000E8000080FB0024
:101EA4000041880070ED880060BD2800FA26070014
:101EB4000000060030E62100104078000004E00035
:101EC40004003A000017280001002000B532070082
:101ED400110037000080FB00010320000180B900DD
:101EE4002002B000E1A92100610078000000010097
:101EF4004045280001002000AA320700C002A900C2
:101F0400C202A900204628000100200079320700FF
:101F140060BD2800E02607000000060030E621002E
:101F24001004E00004003A0000172800010020001B
:101F34009C3207002B003700C002A900C202A8008F
:101F440021E3A8002000200034250700A000200081
:101F540005250700011B2000810F500016003600E4
:101F64009000200000250700712B2000810F5000F5
:101F740011003600A0552800010020005D32070042
:101F840060BD2800C426070030E621009080FB00D5
:101F9400000320000088B9000002B000E1A921007C
:101FA4006100780000000100605328000100200057
:101FB4007C3207000A003700C002A900C202A9004F
:101FC4002013280001002000763207002046280054
:101FD400010020004732070060BD2800AE2607003C
:101FE40021E3A90000000600889FBE008A9FBE006E
:101FF40071ED8000004180008004EB00808F500070
:102004000E003200EACA21000BC2B3000104E8004A
:102014006A407C0000F578000004E00001003A000A
:102024000B4078007B2507008904E8008880FB00CA
:1020340000418000810F5000F4FF3A000000E900E5
:102044000080FB000041880070BD280025260700A1
:1020540009007800E0250700A0BD2800212607001C
:102064004F05BE004F04BE000000060070ED800066
:102074002208E30003003A0070C0B300652507009E
:10208400150037002008E3000B003A000000E900C7
:102094000080FB00004188000041EB00E1CA210000
:1020A4008270780070ED8800608E280001002000A6
:1020B4001032070008003700A08D2800010020001E
:1020C4000C320700E0DA21001001E900F10F2000D2
:1020D40001086100C4FF07000000060070ED8000E5
:1020E4002208E30003003A0070C0B300492507004A
:1020F40001003700BCFF070000000600889FBE00F7
:1021040070ED80002208E30002003A0070C0B300C2
:1021140040250700E9DA2100184180001904140061
:102124000884FB0070BD2800EE2507000800780035
:10213400A9250700A0BD2800EA250700104180005A
:10214400800C78004F04BE0000000600889FBE008B
:1021540070ED80002008E30002003A0070C0B30074
:102164002C250700E9DA21000841800019045400F5
:102174000884FB0070BD2800DA25070008007800F9
:1021840095250700C0BD2800D62507000041800022
:10219400800C78004F04BE0000000600889FBE003B
:1021A4008A9FBE008C9FBE008E1F780080467800F8
:1021B4000A4180000A00E8000080FB002208E300D6
:1021C40044003200FFCF560042003600E0C7B3009F
:1021D40080CF56003F003E0078ED8000880F550008
:1021E4000C003A000D4078000A25070000418000E9
:1021F400E1CA21008D7078000000E8000080FB0037
:10220400004188000041EB008270780070ED880086
:102214003200370070BD2800B225070008045500BD
:10222400FB0F20000B0064006B250700C0BD2800D5
:10223400AC2507000A418000E0DA21001000E90023
:102244008B0560008A8F550014003200EBCA210010
:10225400E88D280009002000FC0F2000EEDA2100A0
:102264000A804500EB407D00114098006B407D00E2
:102274000004E00003003200E62407000800BE006A
:102284009C3107000A05E9000C0565001E00E90001
:102294000C0060008A0F5000F1FF3A000D407800F6
:1022A400DC240700E1DA210011007800E2CA2100F1
:1022B4000D7178000001E800F00F20008008610033
:1022C400014180008100E800008160000241880033
:1022D4000200370070C0B300CE2407004F07780017
:1022E4004F06BE004F05BE004F04BE0000000600AE
:1022F40020DB210041C0B30090CF10000400360061
:102304006C31070020DB21000048EB000D00370092
:1023140070ED80002208E300080032000000E900AC
:10232400F20F2000E1DA210082086000A08D28006D
:10233400010020006F3107000200370070C0B300B5
:10234400B424070000000600AE240700B1C5B300A2
:10235400814F500026003A00AA24070011C4B3009C
:10236400814F50001300320007003E00F0C05000BF
:10237400814F500013003200E3C04000814F5000F1
:102384001B003A001500370031C4B300814F5000E0
:1023940006003200090039008140E800814F5000F6
:1023A40013003A00D2FF070011003700ECFD0700CC
:1023B4000F0037004FFE07000D00370071FE0700C5
:1023C4000B0037008F240700E1C7B300814F500092
:1023D40007003A0049FF0700050037008924070079
:1023E400E1C7B300814F500001003A0057FF0700D6
:1023F40000000600889FBE00C07328000100200072
:1024040068310700E0AC27000100200065310700B7
:10241400E02B2800010020003631070030E62100BF
:102424009080FB00000320000088B9004002B00047
:10243400E1A9210061007800000001004074280037
:10244400010020002B31070000402000AFFD0700F1
:1024540000102000ADFD070000202000ABFD0700A8
:1024640000042000A9FD070000082000A7FD0700C4
:1024740060BD280088250700E08B280001002000AB
:102484001C31070021E3A800A0002000B6230700A8
:10249400DC24070088942800090020000800BE00FE
:1024A4001431070090C0B3005A24070090002000A4
:1024B400AD230700D32407000800BE000D31070038
:1024C40090C0B30053240700C0002000A6230700D7
:1024D400CC2407000800BE000631070090C0B300FA
:1024E4004C240700B00020009F230700C5240700E8
:1024F4000800BE00FF30070090C0B3004524070069
:1025040021E3A9000040200087FD070000102000FF
:1025140085FD07000020200083FD07000004200043
:1025240081FD0700000820007FFD070060BD280032
:10253400592507004F04BE000000060060882800EB
:1025440001002000EB300700C1BF2A000000EB00AF
:10255400A12307003A240700407F2800010020003F
:10256400E4300700E1BF2A000000EB009A230700D3
:102574003324070060BD28004725070000622800B7
:1025840001002000073107009AFF0700C202AB00D8
:1025940004003200A055280001002000D5300700B7
:1025A400030037002046280001002000D130070036
:1025B400C0C2B3001724070000C2B30015240700EB
:1025C400CB62AB0004003200403E28000100200032
:1025D400C830070003003700403228000100200003
:1025E400C4300700C0C2B3000A24070000C2B3000D
:1025F4000824070080E62100104078007040600045
:102604000400320020F6270001002000E530070016
:1026140003003700E00A280001002000E130070031
:1026240080E62100104078006840600004003A0011
:102634004018280001002000AE30070003003700D6
:102644008019280001002000AA300700C0C2B3008E
:10265400F023070000C2B300EE230700401D28004A
:1026640001002000A330070070E62100104078002C
:102674005224070060BD28000725070080E62100DA
:102684001040780063406000E14F500004003A00BD
:102694004031280001002000C23007000300370049
:1026A4004030280001002000BE30070030E6210041
:1026B4009080FB00000320000088B9006002B00095
:1026C400E1A92100610078000000010000622800F7
:1026D40001002000B330070000000600889FBE0000
:1026E4008A9FBE00134180000380FB00E1CA2100E1
:1026F40061407800F1CCB30081404000E8CF500045
:102704001A003E000000FB000003B1008300E80053
:102714008180FB00E2CA210062C1780004CDB300CD
:102724000442410011002000E94F520076003E00AF
:10273400F80F2000E7CA210006CDB3006A02B900F1
:102744000200FB00040040000003B1008100E80027
:10275400038140000801610067417900064241009D
:10276400E94F5200F5FF36006700370001C3B3009C
:10277400814F500060003A000300E8000080FB0035
:10278400E1CA21006141780020C6B300804F5100A6
:102794000B003A000380E8000080FB00E1CA21003E
:1027A4006141780004CDB300044241000000EB0015
:1027B40021002000E14F520005003600520037008E
:1027C40020C4B300804F510010003A00F1FF3700DD
:1027D400F70F2000E6CA210005CDB3000000400039
:1027E4000201FB00020040000003B1008100E80088
:1027F4000381400007016100664179000542410000
:10280400E14F5200F5FF36003F00370080C7B300A8
:10281400804F51000A00320080C5B300804F510040
:102824001E003A00090037004400DD000003B10037
:102834000201FB00020040008100E8000A003700AA
:102844000000EB0021002000020037000000EB0034
:1028540021002000F90F2000E7CA210008CDB300B1
:10286400FACBB300FBC9B300038240000902620043
:1028740067417A0088424100E9CF5200EAFF3600FE
:102884008A424100E5CF5200260036000B43410046
:10289400E54F5300230036001B00370004CDB3007E
:1028A400044241000000EB0011002000E94F5200F7
:1028B40015003E000200FB000003B100F80F2000E9
:1028C400E7CA210006CDB3006A02B9000200FB008A
:1028D400040040000003B1008100E80003814000CF
:1028E400080161006741790006424100E94F520046
:1028F400F5FF36000400370080E621001074A000C4
:102904000000EB00040037002282200092C0400047
:102914008180FB00114188004F05BE004F04BE00BA
:10292400000006000254A00082737A004400DD0017
:102934007005B1000201FB0002004000BEFF370039
:10294400881F7800114180000100E8000080FB002E
:10295400E2CA2100E241780010002000A2C3B300C3
:1029640082CF510009003A008180E800F80F20006E
:10297400088060001041880058FF07001141800062
:102984008100E90008816000124188004F0478004A
:1029940000000600881F7800114180000100E80053
:1029A4000080FB00E2CA2100E24178000000EB0055
:1029B400B2C3B30082CF510009003A008180E8001D
:1029C400F80F2000088060001041880043FF0700D2
:1029D400114180008100E9000881600012418800F3
:1029E4004F0478000000060010418000E1CA210075
:1029F4006141780001C2B300814F510009003A00DF
:102A0400F40F2000E3CA2100014178000000E8002F
:102A140004006000E340780082CF5000FBFF3200E6
:102A24001041880000000600889FBE008A1F7800BD
:102A3400004478002208EC000080FB00104188006C
:102A4400E9FF070025FF0700000578000804E000FF
:102A54000500320070E62100904078000A007800FA
:102A640048220700000578000A4078000A2307007E
:102A7400A88C2800090020000800BE009D2F070034
:102A84000A4078004D2307000800BE00992F070074
:102A94000A4078007A23070060BD2800FE2307005F
:102AA4004F0578004F04BE0000000600F28747007F
:102AB400889FBE008A9FBE008C9FBE008E1F780038
:102AC400E0B79F00D1B79F00C2B79F00F3B79F0044
:102AD4000ECDB300688E280009002000CA1A280011
:102AE4000B002000E0BD28007E2307006FB0970094
:102AF4000000E00003003D0020BE28007923070009
:102B0400020037004FE897002C23070040BE28003E
:102B1400742307008000EB0081BF9F008006EB0058
:102B2400B822070000467800ED4F50003E00320006
:102B340005003C00E84F50000A003200EA4F500004
:102B440026003A0038003700D1C2B300814F50004C
:102B54001500320081C7B300814F50001F003A00B6
:102B64001B0037000D00E000040032008D06E90070
:102B74000800BE005F2F0700E9FF37000FB9970078
:102B84000200E000050032000800BE00592F0700D3
:102B94000000EB0080BF9F00E1FF370070C0B3006E
:102BA4009C220700DEFF37000D00E00005003A001C
:102BB400D0C2B300972207001100200081BF9F00FC
:102BC400D7FF370070C0B30092220700D4FF37004C
:102BD4007FB197000200E00031003A000E4040004F
:102BE400E94F50000D003E00E38F5600040034000E
:102BF40070C0B300872207004D002000C8FF3700D3
:102C04000C407800832207008C4078007E805700B7
:102C140001F07E008D06E800C1FF370070C0B300EC
:102C24007C220700BEFF370060BD28009A230700FE
:102C34000D00E0001E0032000D00E9008000EB00F2
:102C4400080033007E8057008D0640006A09B900F1
:102C5400B000FB000103B100828040008D0F5000E2
:102C6400FAFF3A005FB19700810F510009003C0060
:102C74004FB09700810F5000060035000FB9970040
:102C84000200E000090032000100EA00E0B79F0002
:102C9400070037000A00BE00422F070091FF3700EB
:102CA4000080EB00E0B79F0001003700E1B79F0010
:102CB4006FB097004F0778004F06BE004F05BE0067
:102CC4004F04BE002F01B100000006000E00FA0000
:102CD400889FBE008A9FBE008C9FBE00104180006A
:102CE4000004E9000884FB001D002000880F500048
:102CF40026003200E9CA2100FB0F200069407C0055
:102D04000004E0001C003A000806E8000B06660018
:102D140069407E000004E000170032000D40780096
:102D2400A622070070BE2800EE22070069407E003C
:102D34000004E000070032000885E800352207009F
:102D44000B006500694078000A05E8000004E00013
:102D5400FAFF3A000D8046000C017800FA80570013
:102D6400823078008D06E800E78F560007003200B5
:102D740060BD2800482307000804E9000B04640030
:102D840010418000880F5000DCFF3A0060BD28002D
:102D940041230700807E280001002000012F070046
:102DA400130020000D017800830078000000EB0080
:102DB4003EFF07008000E800E18F50000A00360063
:102DC40000004000FA805700E10278000580FB0013
:102DD400E1CA2100E14078000000EB000104E000BA
